:02000000800B73
:20000B000167758125758902758C2275A882752300752400D28C438701E523B40CF82096C0
:20002B0029E59054E06322FF4522F590D295E5B054C06321FF4521F5B0A2009297C2B7741D
:20004B0096115FD2B775230080CCE590F4541FB522C480DA7F31DFFED5E0F922C0E0C0D0C4
:20006B00C082C0839000C0A295B3E5243393F524B4210B752300752200752100802EB42A9D
:20008B0004D2018005B43224C2010523E523B40106A20192008015C394075009A201E52216
:2000AB0033F5228007A201E52133F521D083D082D0D0D0E032010002000300040005000636
:2000CB00000700080009000A000B000C000D000E000F00100011001200130014001415002F
:2000EB001600171A181A191A001B001C001D1F1E1F001F002000212322232B242B2500260C
:1B010B0028272800280029002A2322232C002D302E302F300031003200222B89
:00000001FF
